:1000000075C6F075C7D875CAE075CBB175C1807576
:10001000C81190F8037492F090F8027400F075F82B
:1000200000780079007A007B00E8C3B4FF00400349
:1000300009800308800012007CEAB499004009EBB3
:100040002401D4FB7A008007EA2401D4FA8000124C
:10005000005480D5EBC4540F2430120084EB540FAD
:100060002430120084EAC4540F2430120084EA546D
:100070000F243012008474201200842288F890F833
:0C00800002E9F022F599C2993099FD22A6
:00000001FF
